
D:\STM32\Program\1.11_Odchudzanie\um0427\FWLib\project\RIDE\STM3210E-EVAL\t6963c.o:     file format elf32-littlearm
D:\STM32\Program\1.11_Odchudzanie\um0427\FWLib\project\RIDE\STM3210E-EVAL\t6963c.o

Disassembly of section .text.delay:

00000000 <delay>:
delay():
D:\STM32\Program\1.11_Odchudzanie\um0427\FWLib\project/t6963c.c:10
   0:	b082      	sub	sp, #8
D:\STM32\Program\1.11_Odchudzanie\um0427\FWLib\project/t6963c.c:12
   2:	2300      	movs	r3, #0
   4:	e002      	b.n	c <delay+0xc>
D:\STM32\Program\1.11_Odchudzanie\um0427\FWLib\project/t6963c.c:13
   6:	bf00      	nop
D:\STM32\Program\1.11_Odchudzanie\um0427\FWLib\project/t6963c.c:12
   8:	9b01      	ldr	r3, [sp, #4]
   a:	3301      	adds	r3, #1
   c:	9301      	str	r3, [sp, #4]
   e:	9b01      	ldr	r3, [sp, #4]
  10:	2b0a      	cmp	r3, #10
  12:	ddf8      	ble.n	6 <delay+0x6>
D:\STM32\Program\1.11_Odchudzanie\um0427\FWLib\project/t6963c.c:15
  14:	b002      	add	sp, #8
  16:	4770      	bx	lr
Disassembly of section .text.outByte:

00000000 <outByte>:
outByte():
D:\STM32\Program\1.11_Odchudzanie\um0427\FWLib\project/t6963c.c:20
   0:	b570      	push	{r4, r5, r6, lr}
D:\STM32\Program\1.11_Odchudzanie\um0427\FWLib\project/t6963c.c:21
   2:	4c0e      	ldr	r4, [pc, #56]	(3c <outByte+0x3c>)
D:\STM32\Program\1.11_Odchudzanie\um0427\FWLib\project/t6963c.c:24
   4:	4d0e      	ldr	r5, [pc, #56]	(40 <outByte+0x40>)
D:\STM32\Program\1.11_Odchudzanie\um0427\FWLib\project/t6963c.c:20
   6:	4606      	mov	r6, r0
D:\STM32\Program\1.11_Odchudzanie\um0427\FWLib\project/t6963c.c:21
   8:	4620      	mov	r0, r4
   a:	f7ff fffe 	bl	0 <GPIO_StructInit>
D:\STM32\Program\1.11_Odchudzanie\um0427\FWLib\project/t6963c.c:22
   e:	f64f 7300 	movw	r3, #65280	; 0xff00
D:\STM32\Program\1.11_Odchudzanie\um0427\FWLib\project/t6963c.c:24
  12:	4628      	mov	r0, r5
  14:	4621      	mov	r1, r4
D:\STM32\Program\1.11_Odchudzanie\um0427\FWLib\project/t6963c.c:22
  16:	8023      	strh	r3, [r4, #0]
D:\STM32\Program\1.11_Odchudzanie\um0427\FWLib\project/t6963c.c:23
  18:	2310      	movs	r3, #16
  1a:	70e3      	strb	r3, [r4, #3]
D:\STM32\Program\1.11_Odchudzanie\um0427\FWLib\project/t6963c.c:24
  1c:	f7ff fffe 	bl	0 <GPIO_Init>
D:\STM32\Program\1.11_Odchudzanie\um0427\FWLib\project/t6963c.c:26
  20:	f7ff fffe 	bl	0 <outByte>
D:\STM32\Program\1.11_Odchudzanie\um0427\FWLib\project/t6963c.c:27
  24:	0231      	lsls	r1, r6, #8
  26:	4628      	mov	r0, r5
D:\STM32\Program\1.11_Odchudzanie\um0427\FWLib\project/t6963c.c:29
  28:	0236      	lsls	r6, r6, #8
D:\STM32\Program\1.11_Odchudzanie\um0427\FWLib\project/t6963c.c:27
  2a:	f7ff fffe 	bl	0 <GPIO_SetBits>
D:\STM32\Program\1.11_Odchudzanie\um0427\FWLib\project/t6963c.c:29
  2e:	4628      	mov	r0, r5
  30:	f486 417f 	eor.w	r1, r6, #65280	; 0xff00
  34:	f7ff fffe 	bl	0 <GPIO_ResetBits>
D:\STM32\Program\1.11_Odchudzanie\um0427\FWLib\project/t6963c.c:31
  38:	bd70      	pop	{r4, r5, r6, pc}
  3a:	46c0      	nop			(mov r8, r8)
  3c:	00000000 	.word	0x00000000
  40:	40010c00 	.word	0x40010c00
Disassembly of section .text.inByte:

00000000 <inByte>:
inByte():
D:\STM32\Program\1.11_Odchudzanie\um0427\FWLib\project/t6963c.c:35
   0:	b570      	push	{r4, r5, r6, lr}
D:\STM32\Program\1.11_Odchudzanie\um0427\FWLib\project/t6963c.c:37
   2:	4c0b      	ldr	r4, [pc, #44]	(30 <inByte+0x30>)
D:\STM32\Program\1.11_Odchudzanie\um0427\FWLib\project/t6963c.c:40
   4:	4d0b      	ldr	r5, [pc, #44]	(34 <inByte+0x34>)
D:\STM32\Program\1.11_Odchudzanie\um0427\FWLib\project/t6963c.c:37
   6:	4620      	mov	r0, r4
   8:	f7ff fffe 	bl	0 <GPIO_StructInit>
D:\STM32\Program\1.11_Odchudzanie\um0427\FWLib\project/t6963c.c:38
   c:	f64f 7300 	movw	r3, #65280	; 0xff00
D:\STM32\Program\1.11_Odchudzanie\um0427\FWLib\project/t6963c.c:40
  10:	4628      	mov	r0, r5
  12:	4621      	mov	r1, r4
D:\STM32\Program\1.11_Odchudzanie\um0427\FWLib\project/t6963c.c:38
  14:	8023      	strh	r3, [r4, #0]
D:\STM32\Program\1.11_Odchudzanie\um0427\FWLib\project/t6963c.c:39
  16:	2348      	movs	r3, #72
  18:	70e3      	strb	r3, [r4, #3]
D:\STM32\Program\1.11_Odchudzanie\um0427\FWLib\project/t6963c.c:40
  1a:	f7ff fffe 	bl	0 <GPIO_Init>
D:\STM32\Program\1.11_Odchudzanie\um0427\FWLib\project/t6963c.c:42
  1e:	f7ff fffe 	bl	0 <inByte>
D:\STM32\Program\1.11_Odchudzanie\um0427\FWLib\project/t6963c.c:43
  22:	4628      	mov	r0, r5
  24:	f7ff fffe 	bl	0 <GPIO_ReadInputData>
D:\STM32\Program\1.11_Odchudzanie\um0427\FWLib\project/t6963c.c:46
  28:	f3c0 2007 	ubfx	r0, r0, #8, #8
  2c:	bd70      	pop	{r4, r5, r6, pc}
  2e:	46c0      	nop			(mov r8, r8)
  30:	00000000 	.word	0x00000000
  34:	40010c00 	.word	0x40010c00
Disassembly of section .text.GLCD_Chceck_Status:

00000000 <GLCD_Chceck_Status>:
GLCD_Chceck_Status():
D:\STM32\Program\1.11_Odchudzanie\um0427\FWLib\project/t6963c.c:50
   0:	b570      	push	{r4, r5, r6, lr}
D:\STM32\Program\1.11_Odchudzanie\um0427\FWLib\project/t6963c.c:55
   2:	4c11      	ldr	r4, [pc, #68]	(48 <GLCD_Chceck_Status+0x48>)
D:\STM32\Program\1.11_Odchudzanie\um0427\FWLib\project/t6963c.c:54
   4:	2140      	movs	r1, #64
   6:	4811      	ldr	r0, [pc, #68]	(4c <GLCD_Chceck_Status+0x4c>)
   8:	f7ff fffe 	bl	0 <GPIO_SetBits>
D:\STM32\Program\1.11_Odchudzanie\um0427\FWLib\project/t6963c.c:57
   c:	4d10      	ldr	r5, [pc, #64]	(50 <GLCD_Chceck_Status+0x50>)
D:\STM32\Program\1.11_Odchudzanie\um0427\FWLib\project/t6963c.c:55
   e:	4620      	mov	r0, r4
  10:	2140      	movs	r1, #64
  12:	f7ff fffe 	bl	0 <GPIO_SetBits>
D:\STM32\Program\1.11_Odchudzanie\um0427\FWLib\project/t6963c.c:56
  16:	4620      	mov	r0, r4
  18:	2180      	movs	r1, #128
  1a:	f7ff fffe 	bl	0 <GPIO_ResetBits>
D:\STM32\Program\1.11_Odchudzanie\um0427\FWLib\project/t6963c.c:57
  1e:	4628      	mov	r0, r5
  20:	f44f 7180 	mov.w	r1, #256	; 0x100
  24:	f7ff fffe 	bl	0 <GPIO_ResetBits>
D:\STM32\Program\1.11_Odchudzanie\um0427\FWLib\project/t6963c.c:58
  28:	f7ff fffe 	bl	0 <GLCD_Chceck_Status>
D:\STM32\Program\1.11_Odchudzanie\um0427\FWLib\project/t6963c.c:60
  2c:	f7ff fffe 	bl	0 <GLCD_Chceck_Status>
D:\STM32\Program\1.11_Odchudzanie\um0427\FWLib\project/t6963c.c:62
  30:	f44f 7180 	mov.w	r1, #256	; 0x100
D:\STM32\Program\1.11_Odchudzanie\um0427\FWLib\project/t6963c.c:60
  34:	4606      	mov	r6, r0
D:\STM32\Program\1.11_Odchudzanie\um0427\FWLib\project/t6963c.c:62
  36:	4628      	mov	r0, r5
  38:	f7ff fffe 	bl	0 <GPIO_SetBits>
D:\STM32\Program\1.11_Odchudzanie\um0427\FWLib\project/t6963c.c:63
  3c:	4620      	mov	r0, r4
  3e:	2180      	movs	r1, #128
  40:	f7ff fffe 	bl	0 <GPIO_SetBits>
D:\STM32\Program\1.11_Odchudzanie\um0427\FWLib\project/t6963c.c:66
  44:	4630      	mov	r0, r6
  46:	bd70      	pop	{r4, r5, r6, pc}
  48:	40011000 	.word	0x40011000
  4c:	40010c00 	.word	0x40010c00
  50:	40010800 	.word	0x40010800
Disassembly of section .text.GLCD_Read_Data:

00000000 <GLCD_Read_Data>:
GLCD_Read_Data():
D:\STM32\Program\1.11_Odchudzanie\um0427\FWLib\project/t6963c.c:103
   0:	b510      	push	{r4, lr}
D:\STM32\Program\1.11_Odchudzanie\um0427\FWLib\project/t6963c.c:105
   2:	f7ff fffe 	bl	0 <GLCD_Read_Data>
   6:	f010 0f03 	tst.w	r0, #3	; 0x3
   a:	d0fa      	beq.n	2 <GLCD_Read_Data+0x2>
D:\STM32\Program\1.11_Odchudzanie\um0427\FWLib\project/t6963c.c:107
   c:	2140      	movs	r1, #64
   e:	4810      	ldr	r0, [pc, #64]	(50 <GLCD_Read_Data+0x50>)
  10:	f7ff fffe 	bl	0 <GPIO_ResetBits>
D:\STM32\Program\1.11_Odchudzanie\um0427\FWLib\project/t6963c.c:108
  14:	2140      	movs	r1, #64
  16:	480f      	ldr	r0, [pc, #60]	(54 <GLCD_Read_Data+0x54>)
  18:	f7ff fffe 	bl	0 <GPIO_SetBits>
D:\STM32\Program\1.11_Odchudzanie\um0427\FWLib\project/t6963c.c:109
  1c:	2180      	movs	r1, #128
  1e:	480d      	ldr	r0, [pc, #52]	(54 <GLCD_Read_Data+0x54>)
  20:	f7ff fffe 	bl	0 <GPIO_ResetBits>
D:\STM32\Program\1.11_Odchudzanie\um0427\FWLib\project/t6963c.c:110
  24:	f44f 7180 	mov.w	r1, #256	; 0x100
  28:	480b      	ldr	r0, [pc, #44]	(30 <GPIO_ResetBits+0x30>)
  2a:	f7ff fffe 	bl	0 <GPIO_ResetBits>
D:\STM32\Program\1.11_Odchudzanie\um0427\FWLib\project/t6963c.c:112
  2e:	f7ff fffe 	bl	0 <GLCD_Read_Data>
D:\STM32\Program\1.11_Odchudzanie\um0427\FWLib\project/t6963c.c:113
  32:	f7ff fffe 	bl	0 <GLCD_Read_Data>
D:\STM32\Program\1.11_Odchudzanie\um0427\FWLib\project/t6963c.c:114
  36:	f44f 7180 	mov.w	r1, #256	; 0x100
D:\STM32\Program\1.11_Odchudzanie\um0427\FWLib\project/t6963c.c:113
  3a:	4604      	mov	r4, r0
D:\STM32\Program\1.11_Odchudzanie\um0427\FWLib\project/t6963c.c:114
  3c:	4806      	ldr	r0, [pc, #24]	(58 <GLCD_Read_Data+0x58>)
  3e:	f7ff fffe 	bl	0 <GPIO_SetBits>
D:\STM32\Program\1.11_Odchudzanie\um0427\FWLib\project/t6963c.c:115
  42:	4804      	ldr	r0, [pc, #16]	(54 <GLCD_Read_Data+0x54>)
  44:	2180      	movs	r1, #128
  46:	f7ff fffe 	bl	0 <GPIO_SetBits>
D:\STM32\Program\1.11_Odchudzanie\um0427\FWLib\project/t6963c.c:118
  4a:	4620      	mov	r0, r4
  4c:	bd10      	pop	{r4, pc}
  4e:	46c0      	nop			(mov r8, r8)
  50:	40010c00 	.word	0x40010c00
  54:	40011000 	.word	0x40011000
  58:	40010800 	.word	0x40010800
Disassembly of section .text.GLCD_Write_Data:

00000000 <GLCD_Write_Data>:
GLCD_Write_Data():
D:\STM32\Program\1.11_Odchudzanie\um0427\FWLib\project/t6963c.c:87
   0:	b510      	push	{r4, lr}
   2:	4604      	mov	r4, r0
D:\STM32\Program\1.11_Odchudzanie\um0427\FWLib\project/t6963c.c:88
   4:	f7ff fffe 	bl	0 <GLCD_Write_Data>
   8:	f010 0f03 	tst.w	r0, #3	; 0x3
   c:	d0fa      	beq.n	4 <GLCD_Write_Data+0x4>
D:\STM32\Program\1.11_Odchudzanie\um0427\FWLib\project/t6963c.c:90
   e:	b2e0      	uxtb	r0, r4
  10:	f7ff fffe 	bl	0 <GLCD_Write_Data>
D:\STM32\Program\1.11_Odchudzanie\um0427\FWLib\project/t6963c.c:91
  14:	2140      	movs	r1, #64
  16:	480e      	ldr	r0, [pc, #56]	(50 <GLCD_Write_Data+0x50>)
  18:	f7ff fffe 	bl	0 <GPIO_ResetBits>
D:\STM32\Program\1.11_Odchudzanie\um0427\FWLib\project/t6963c.c:92
  1c:	2180      	movs	r1, #128
  1e:	480d      	ldr	r0, [pc, #52]	(54 <GLCD_Write_Data+0x54>)
  20:	f7ff fffe 	bl	0 <GPIO_SetBits>
D:\STM32\Program\1.11_Odchudzanie\um0427\FWLib\project/t6963c.c:93
  24:	2140      	movs	r1, #64
  26:	480b      	ldr	r0, [pc, #44]	(54 <GLCD_Write_Data+0x54>)
  28:	f7ff fffe 	bl	0 <GPIO_ResetBits>
D:\STM32\Program\1.11_Odchudzanie\um0427\FWLib\project/t6963c.c:94
  2c:	480a      	ldr	r0, [pc, #40]	(58 <GLCD_Write_Data+0x58>)
  2e:	f44f 7180 	mov.w	r1, #256	; 0x100
  32:	f7ff fffe 	bl	0 <GPIO_ResetBits>
D:\STM32\Program\1.11_Odchudzanie\um0427\FWLib\project/t6963c.c:96
  36:	f7ff fffe 	bl	0 <GLCD_Write_Data>
D:\STM32\Program\1.11_Odchudzanie\um0427\FWLib\project/t6963c.c:97
  3a:	4807      	ldr	r0, [pc, #28]	(58 <GLCD_Write_Data+0x58>)
  3c:	f44f 7180 	mov.w	r1, #256	; 0x100
  40:	f7ff fffe 	bl	0 <GPIO_SetBits>
D:\STM32\Program\1.11_Odchudzanie\um0427\FWLib\project/t6963c.c:98
  44:	4803      	ldr	r0, [pc, #12]	(54 <GLCD_Write_Data+0x54>)
  46:	2140      	movs	r1, #64
  48:	f7ff fffe 	bl	0 <GPIO_SetBits>
D:\STM32\Program\1.11_Odchudzanie\um0427\FWLib\project/t6963c.c:100
  4c:	bd10      	pop	{r4, pc}
  4e:	46c0      	nop			(mov r8, r8)
  50:	40010c00 	.word	0x40010c00
  54:	40011000 	.word	0x40011000
  58:	40010800 	.word	0x40010800
Disassembly of section .text.GLCD_Write_Command:

00000000 <GLCD_Write_Command>:
GLCD_Write_Command():
D:\STM32\Program\1.11_Odchudzanie\um0427\FWLib\project/t6963c.c:70
   0:	b510      	push	{r4, lr}
   2:	4604      	mov	r4, r0
D:\STM32\Program\1.11_Odchudzanie\um0427\FWLib\project/t6963c.c:71
   4:	f7ff fffe 	bl	0 <GLCD_Write_Command>
   8:	f010 0f03 	tst.w	r0, #3	; 0x3
   c:	d0fa      	beq.n	4 <GLCD_Write_Command+0x4>
D:\STM32\Program\1.11_Odchudzanie\um0427\FWLib\project/t6963c.c:73
   e:	b2e0      	uxtb	r0, r4
  10:	f7ff fffe 	bl	0 <GLCD_Write_Command>
D:\STM32\Program\1.11_Odchudzanie\um0427\FWLib\project/t6963c.c:75
  14:	2140      	movs	r1, #64
  16:	480c      	ldr	r0, [pc, #48]	(48 <GLCD_Write_Command+0x48>)
  18:	f7ff fffe 	bl	0 <GPIO_SetBits>
D:\STM32\Program\1.11_Odchudzanie\um0427\FWLib\project/t6963c.c:76
  1c:	2140      	movs	r1, #64
  1e:	480b      	ldr	r0, [pc, #44]	(4c <GLCD_Write_Command+0x4c>)
  20:	f7ff fffe 	bl	0 <GPIO_ResetBits>
D:\STM32\Program\1.11_Odchudzanie\um0427\FWLib\project/t6963c.c:77
  24:	480a      	ldr	r0, [pc, #40]	(50 <GLCD_Write_Command+0x50>)
  26:	f44f 7180 	mov.w	r1, #256	; 0x100
  2a:	f7ff fffe 	bl	0 <GPIO_ResetBits>
D:\STM32\Program\1.11_Odchudzanie\um0427\FWLib\project/t6963c.c:79
  2e:	f7ff fffe 	bl	0 <GLCD_Write_Command>
D:\STM32\Program\1.11_Odchudzanie\um0427\FWLib\project/t6963c.c:81
  32:	2140      	movs	r1, #64
  34:	4805      	ldr	r0, [pc, #20]	(4c <GLCD_Write_Command+0x4c>)
  36:	f7ff fffe 	bl	0 <GPIO_SetBits>
D:\STM32\Program\1.11_Odchudzanie\um0427\FWLib\project/t6963c.c:82
  3a:	4805      	ldr	r0, [pc, #20]	(50 <GLCD_Write_Command+0x50>)
  3c:	f44f 7180 	mov.w	r1, #256	; 0x100
  40:	f7ff fffe 	bl	0 <GPIO_SetBits>
D:\STM32\Program\1.11_Odchudzanie\um0427\FWLib\project/t6963c.c:83
  44:	bd10      	pop	{r4, pc}
  46:	46c0      	nop			(mov r8, r8)
  48:	40010c00 	.word	0x40010c00
  4c:	40011000 	.word	0x40011000
  50:	40010800 	.word	0x40010800
Disassembly of section .text.GLCD_SetPixel:

00000000 <GLCD_SetPixel>:
GLCD_SetPixel():
D:\STM32\Program\1.11_Odchudzanie\um0427\FWLib\project/t6963c.c:324
   0:	e92d 41f0 	stmdb	sp!, {r4, r5, r6, r7, r8, lr}
D:\STM32\Program\1.11_Odchudzanie\um0427\FWLib\project/t6963c.c:328
   4:	2606      	movs	r6, #6
   6:	fb90 f5f6 	sdiv	r5, r0, r6
   a:	f505 7320 	add.w	r3, r5, #640	; 0x280
   e:	2428      	movs	r4, #40
  10:	fb01 3404 	mla	r4, r1, r4, r3
D:\STM32\Program\1.11_Odchudzanie\um0427\FWLib\project/t6963c.c:324
  14:	4607      	mov	r7, r0
D:\STM32\Program\1.11_Odchudzanie\um0427\FWLib\project/t6963c.c:330
  16:	b2e0      	uxtb	r0, r4
D:\STM32\Program\1.11_Odchudzanie\um0427\FWLib\project/t6963c.c:324
  18:	4690      	mov	r8, r2
D:\STM32\Program\1.11_Odchudzanie\um0427\FWLib\project/t6963c.c:330
  1a:	f7ff fffe 	bl	0 <GLCD_SetPixel>
D:\STM32\Program\1.11_Odchudzanie\um0427\FWLib\project/t6963c.c:331
  1e:	1220      	asrs	r0, r4, #8
  20:	f7ff fffe 	bl	0 <GLCD_SetPixel>
D:\STM32\Program\1.11_Odchudzanie\um0427\FWLib\project/t6963c.c:332
  24:	2024      	movs	r0, #36
  26:	f7ff fffe 	bl	0 <GLCD_SetPixel>
D:\STM32\Program\1.11_Odchudzanie\um0427\FWLib\project/t6963c.c:334
  2a:	20c5      	movs	r0, #197
  2c:	f7ff fffe 	bl	0 <GLCD_SetPixel>
D:\STM32\Program\1.11_Odchudzanie\um0427\FWLib\project/t6963c.c:335
  30:	f7ff fffe 	bl	0 <GLCD_SetPixel>
  34:	4601      	mov	r1, r0
  36:	fb05 f006 	mul.w	r0, r5, r6
D:\STM32\Program\1.11_Odchudzanie\um0427\FWLib\project/t6963c.c:337
  3a:	f1b8 0f00 	cmp.w	r8, #0	; 0x0
  3e:	d007      	beq.n	50 <GLCD_SetPixel+0x50>
D:\STM32\Program\1.11_Odchudzanie\um0427\FWLib\project/t6963c.c:338
  40:	1a3a      	subs	r2, r7, r0
  42:	f1c2 0205 	rsb	r2, r2, #5	; 0x5
  46:	2301      	movs	r3, #1
  48:	4093      	lsls	r3, r2
  4a:	ea41 0003 	orr.w	r0, r1, r3
  4e:	e006      	b.n	5e <GLCD_SetPixel+0x5e>
D:\STM32\Program\1.11_Odchudzanie\um0427\FWLib\project/t6963c.c:340
  50:	1a3a      	subs	r2, r7, r0
  52:	f1c2 0205 	rsb	r2, r2, #5	; 0x5
  56:	2301      	movs	r3, #1
  58:	4093      	lsls	r3, r2
  5a:	ea21 0003 	bic.w	r0, r1, r3
D:\STM32\Program\1.11_Odchudzanie\um0427\FWLib\project/t6963c.c:342
  5e:	f7ff fffe 	bl	0 <GLCD_SetPixel>
D:\STM32\Program\1.11_Odchudzanie\um0427\FWLib\project/t6963c.c:343
  62:	20c0      	movs	r0, #192
  64:	f7ff fffe 	bl	0 <GLCD_SetPixel>
D:\STM32\Program\1.11_Odchudzanie\um0427\FWLib\project/t6963c.c:344
  68:	e8bd 81f0 	ldmia.w	sp!, {r4, r5, r6, r7, r8, pc}
Disassembly of section .text.GLCD_Write8Pixels:

00000000 <GLCD_Write8Pixels>:
GLCD_Write8Pixels():
D:\STM32\Program\1.11_Odchudzanie\um0427\FWLib\project/t6963c.c:317
   0:	b510      	push	{r4, lr}
D:\STM32\Program\1.11_Odchudzanie\um0427\FWLib\project/t6963c.c:318
   2:	f7ff fffe 	bl	0 <GLCD_Write8Pixels>
D:\STM32\Program\1.11_Odchudzanie\um0427\FWLib\project/t6963c.c:319
   6:	20c0      	movs	r0, #192
   8:	f7ff fffe 	bl	0 <GLCD_Write8Pixels>
D:\STM32\Program\1.11_Odchudzanie\um0427\FWLib\project/t6963c.c:320
   c:	bd10      	pop	{r4, pc}
   e:	46c0      	nop			(mov r8, r8)
Disassembly of section .text.GLCD_GoTo:

00000000 <GLCD_GoTo>:
GLCD_GoTo():
D:\STM32\Program\1.11_Odchudzanie\um0427\FWLib\project/t6963c.c:309
   0:	2306      	movs	r3, #6
   2:	fbb0 f0f3 	udiv	r0, r0, r3
D:\STM32\Program\1.11_Odchudzanie\um0427\FWLib\project/t6963c.c:305
   6:	b510      	push	{r4, lr}
D:\STM32\Program\1.11_Odchudzanie\um0427\FWLib\project/t6963c.c:309
   8:	f500 7020 	add.w	r0, r0, #640	; 0x280
   c:	2428      	movs	r4, #40
   e:	fb01 0404 	mla	r4, r1, r4, r0
D:\STM32\Program\1.11_Odchudzanie\um0427\FWLib\project/t6963c.c:311
  12:	b2e0      	uxtb	r0, r4
  14:	f7ff fffe 	bl	0 <GLCD_GoTo>
D:\STM32\Program\1.11_Odchudzanie\um0427\FWLib\project/t6963c.c:312
  18:	0a20      	lsrs	r0, r4, #8
  1a:	f7ff fffe 	bl	0 <GLCD_GoTo>
D:\STM32\Program\1.11_Odchudzanie\um0427\FWLib\project/t6963c.c:313
  1e:	2024      	movs	r0, #36
  20:	f7ff fffe 	bl	0 <GLCD_GoTo>
D:\STM32\Program\1.11_Odchudzanie\um0427\FWLib\project/t6963c.c:314
  24:	bd10      	pop	{r4, pc}
  26:	46c0      	nop			(mov r8, r8)
Disassembly of section .text.GLCD_Define_Character:

00000000 <GLCD_Define_Character>:
GLCD_Define_Character():
D:\STM32\Program\1.11_Odchudzanie\um0427\FWLib\project/t6963c.c:288
   0:	b570      	push	{r4, r5, r6, lr}
D:\STM32\Program\1.11_Odchudzanie\um0427\FWLib\project/t6963c.c:292
   2:	00c4      	lsls	r4, r0, #3
   4:	f504 5480 	add.w	r4, r4, #4096	; 0x1000
D:\STM32\Program\1.11_Odchudzanie\um0427\FWLib\project/t6963c.c:294
   8:	4620      	mov	r0, r4
D:\STM32\Program\1.11_Odchudzanie\um0427\FWLib\project/t6963c.c:288
   a:	460d      	mov	r5, r1
D:\STM32\Program\1.11_Odchudzanie\um0427\FWLib\project/t6963c.c:294
   c:	f7ff fffe 	bl	0 <GLCD_Define_Character>
D:\STM32\Program\1.11_Odchudzanie\um0427\FWLib\project/t6963c.c:295
  10:	1220      	asrs	r0, r4, #8
  12:	f7ff fffe 	bl	0 <GLCD_Define_Character>
D:\STM32\Program\1.11_Odchudzanie\um0427\FWLib\project/t6963c.c:296
  16:	2024      	movs	r0, #36
  18:	f7ff fffe 	bl	0 <GLCD_Define_Character>
  1c:	2400      	movs	r4, #0
D:\STM32\Program\1.11_Odchudzanie\um0427\FWLib\project/t6963c.c:300
  1e:	5960      	ldr	r0, [r4, r5]
  20:	f7ff fffe 	bl	0 <GLCD_Define_Character>
D:\STM32\Program\1.11_Odchudzanie\um0427\FWLib\project/t6963c.c:301
  24:	3404      	adds	r4, #4
  26:	20c0      	movs	r0, #192
  28:	f7ff fffe 	bl	0 <GLCD_Define_Character>
D:\STM32\Program\1.11_Odchudzanie\um0427\FWLib\project/t6963c.c:298
  2c:	2c20      	cmp	r4, #32
  2e:	d1f6      	bne.n	1e <GLCD_Define_Character+0x1e>
D:\STM32\Program\1.11_Odchudzanie\um0427\FWLib\project/t6963c.c:303
  30:	bd70      	pop	{r4, r5, r6, pc}
  32:	46c0      	nop			(mov r8, r8)
Disassembly of section .text.GLCD_Text_GoTo:

00000000 <GLCD_Text_GoTo>:
GLCD_Text_GoTo():
D:\STM32\Program\1.11_Odchudzanie\um0427\FWLib\project/t6963c.c:277
   0:	b510      	push	{r4, lr}
D:\STM32\Program\1.11_Odchudzanie\um0427\FWLib\project/t6963c.c:280
   2:	2428      	movs	r4, #40
   4:	fb01 0404 	mla	r4, r1, r4, r0
D:\STM32\Program\1.11_Odchudzanie\um0427\FWLib\project/t6963c.c:282
   8:	4620      	mov	r0, r4
   a:	f7ff fffe 	bl	0 <GLCD_Text_GoTo>
D:\STM32\Program\1.11_Odchudzanie\um0427\FWLib\project/t6963c.c:283
   e:	1220      	asrs	r0, r4, #8
  10:	f7ff fffe 	bl	0 <GLCD_Text_GoTo>
D:\STM32\Program\1.11_Odchudzanie\um0427\FWLib\project/t6963c.c:284
  14:	2024      	movs	r0, #36
  16:	f7ff fffe 	bl	0 <GLCD_Text_GoTo>
D:\STM32\Program\1.11_Odchudzanie\um0427\FWLib\project/t6963c.c:285
  1a:	bd10      	pop	{r4, pc}
Disassembly of section .text.GLCD_Write_Char:

00000000 <GLCD_Write_Char>:
GLCD_Write_Char():
D:\STM32\Program\1.11_Odchudzanie\um0427\FWLib\project/t6963c.c:264
   0:	3820      	subs	r0, #32
D:\STM32\Program\1.11_Odchudzanie\um0427\FWLib\project/t6963c.c:263
   2:	b510      	push	{r4, lr}
D:\STM32\Program\1.11_Odchudzanie\um0427\FWLib\project/t6963c.c:264
   4:	f7ff fffe 	bl	0 <GLCD_Write_Char>
D:\STM32\Program\1.11_Odchudzanie\um0427\FWLib\project/t6963c.c:265
   8:	20c0      	movs	r0, #192
   a:	f7ff fffe 	bl	0 <GLCD_Write_Char>
D:\STM32\Program\1.11_Odchudzanie\um0427\FWLib\project/t6963c.c:266
   e:	bd10      	pop	{r4, pc}
Disassembly of section .text.GLCD_Write_String:

00000000 <GLCD_Write_String>:
GLCD_Write_String():
D:\STM32\Program\1.11_Odchudzanie\um0427\FWLib\project/t6963c.c:269
   0:	b510      	push	{r4, lr}
   2:	4604      	mov	r4, r0
D:\STM32\Program\1.11_Odchudzanie\um0427\FWLib\project/t6963c.c:270
   4:	e003      	b.n	e <GLCD_Write_String+0xe>
D:\STM32\Program\1.11_Odchudzanie\um0427\FWLib\project/t6963c.c:272
   6:	b240      	sxtb	r0, r0
   8:	3401      	adds	r4, #1
   a:	f7ff fffe 	bl	0 <GLCD_Write_String>
D:\STM32\Program\1.11_Odchudzanie\um0427\FWLib\project/t6963c.c:270
   e:	7820      	ldrb	r0, [r4, #0]
  10:	2800      	cmp	r0, #0
  12:	d1f8      	bne.n	6 <GLCD_Write_String+0x6>
D:\STM32\Program\1.11_Odchudzanie\um0427\FWLib\project/t6963c.c:274
  14:	bd10      	pop	{r4, pc}
  16:	46c0      	nop			(mov r8, r8)
Disassembly of section .text.GLCD_Clear_Graphic:

00000000 <GLCD_Clear_Graphic>:
GLCD_Clear_Graphic():
D:\STM32\Program\1.11_Odchudzanie\um0427\FWLib\project/t6963c.c:249
   0:	b510      	push	{r4, lr}
D:\STM32\Program\1.11_Odchudzanie\um0427\FWLib\project/t6963c.c:251
   2:	2080      	movs	r0, #128
   4:	f7ff fffe 	bl	0 <GLCD_Clear_Graphic>
D:\STM32\Program\1.11_Odchudzanie\um0427\FWLib\project/t6963c.c:252
   8:	2002      	movs	r0, #2
   a:	f7ff fffe 	bl	0 <GLCD_Clear_Graphic>
D:\STM32\Program\1.11_Odchudzanie\um0427\FWLib\project/t6963c.c:253
   e:	2024      	movs	r0, #36
  10:	f7ff fffe 	bl	0 <GLCD_Clear_Graphic>
  14:	2400      	movs	r4, #0
D:\STM32\Program\1.11_Odchudzanie\um0427\FWLib\project/t6963c.c:257
  16:	2000      	movs	r0, #0
  18:	f7ff fffe 	bl	0 <GLCD_Clear_Graphic>
D:\STM32\Program\1.11_Odchudzanie\um0427\FWLib\project/t6963c.c:255
  1c:	3401      	adds	r4, #1
D:\STM32\Program\1.11_Odchudzanie\um0427\FWLib\project/t6963c.c:258
  1e:	20c0      	movs	r0, #192
  20:	f7ff fffe 	bl	0 <GLCD_Clear_Graphic>
D:\STM32\Program\1.11_Odchudzanie\um0427\FWLib\project/t6963c.c:255
  24:	f5b4 5fa0 	cmp.w	r4, #5120	; 0x1400
  28:	d1f5      	bne.n	16 <GLCD_Clear_Graphic+0x16>
D:\STM32\Program\1.11_Odchudzanie\um0427\FWLib\project/t6963c.c:260
  2a:	bd10      	pop	{r4, pc}
Disassembly of section .text.GLCD_Clear_CG:

00000000 <GLCD_Clear_CG>:
GLCD_Clear_CG():
D:\STM32\Program\1.11_Odchudzanie\um0427\FWLib\project/t6963c.c:234
   0:	b510      	push	{r4, lr}
D:\STM32\Program\1.11_Odchudzanie\um0427\FWLib\project/t6963c.c:236
   2:	2000      	movs	r0, #0
   4:	f7ff fffe 	bl	0 <GLCD_Clear_CG>
D:\STM32\Program\1.11_Odchudzanie\um0427\FWLib\project/t6963c.c:237
   8:	2010      	movs	r0, #16
   a:	f7ff fffe 	bl	0 <GLCD_Clear_CG>
D:\STM32\Program\1.11_Odchudzanie\um0427\FWLib\project/t6963c.c:238
   e:	2024      	movs	r0, #36
  10:	f7ff fffe 	bl	0 <GLCD_Clear_CG>
  14:	2400      	movs	r4, #0
D:\STM32\Program\1.11_Odchudzanie\um0427\FWLib\project/t6963c.c:242
  16:	2000      	movs	r0, #0
  18:	f7ff fffe 	bl	0 <GLCD_Clear_CG>
D:\STM32\Program\1.11_Odchudzanie\um0427\FWLib\project/t6963c.c:240
  1c:	3401      	adds	r4, #1
D:\STM32\Program\1.11_Odchudzanie\um0427\FWLib\project/t6963c.c:243
  1e:	20c0      	movs	r0, #192
  20:	f7ff fffe 	bl	0 <GLCD_Clear_CG>
D:\STM32\Program\1.11_Odchudzanie\um0427\FWLib\project/t6963c.c:240
  24:	f5b4 6f00 	cmp.w	r4, #2048	; 0x800
  28:	d1f5      	bne.n	16 <GLCD_Clear_CG+0x16>
D:\STM32\Program\1.11_Odchudzanie\um0427\FWLib\project/t6963c.c:245
  2a:	bd10      	pop	{r4, pc}
Disassembly of section .text.GLCD_Clear_Text:

00000000 <GLCD_Clear_Text>:
GLCD_Clear_Text():
D:\STM32\Program\1.11_Odchudzanie\um0427\FWLib\project/t6963c.c:220
   0:	b510      	push	{r4, lr}
D:\STM32\Program\1.11_Odchudzanie\um0427\FWLib\project/t6963c.c:222
   2:	2000      	movs	r0, #0
   4:	f7ff fffe 	bl	0 <GLCD_Clear_Text>
D:\STM32\Program\1.11_Odchudzanie\um0427\FWLib\project/t6963c.c:223
   8:	2000      	movs	r0, #0
   a:	f7ff fffe 	bl	0 <GLCD_Clear_Text>
D:\STM32\Program\1.11_Odchudzanie\um0427\FWLib\project/t6963c.c:224
   e:	2024      	movs	r0, #36
  10:	f7ff fffe 	bl	0 <GLCD_Clear_Text>
  14:	2400      	movs	r4, #0
D:\STM32\Program\1.11_Odchudzanie\um0427\FWLib\project/t6963c.c:228
  16:	2000      	movs	r0, #0
  18:	f7ff fffe 	bl	0 <GLCD_Clear_Text>
D:\STM32\Program\1.11_Odchudzanie\um0427\FWLib\project/t6963c.c:226
  1c:	3401      	adds	r4, #1
D:\STM32\Program\1.11_Odchudzanie\um0427\FWLib\project/t6963c.c:229
  1e:	20c0      	movs	r0, #192
  20:	f7ff fffe 	bl	0 <GLCD_Clear_Text>
D:\STM32\Program\1.11_Odchudzanie\um0427\FWLib\project/t6963c.c:226
  24:	f5b4 7f20 	cmp.w	r4, #640	; 0x280
  28:	d1f5      	bne.n	16 <GLCD_Clear_Text+0x16>
D:\STM32\Program\1.11_Odchudzanie\um0427\FWLib\project/t6963c.c:231
  2a:	bd10      	pop	{r4, pc}
Disassembly of section .text.GLCD_Ustaw_Adres:

00000000 <GLCD_Ustaw_Adres>:
GLCD_Ustaw_Adres():
D:\STM32\Program\1.11_Odchudzanie\um0427\FWLib\project/t6963c.c:212
   0:	b510      	push	{r4, lr}
   2:	4604      	mov	r4, r0
D:\STM32\Program\1.11_Odchudzanie\um0427\FWLib\project/t6963c.c:213
   4:	b2c0      	uxtb	r0, r0
   6:	f7ff fffe 	bl	0 <GLCD_Ustaw_Adres>
D:\STM32\Program\1.11_Odchudzanie\um0427\FWLib\project/t6963c.c:214
   a:	0a20      	lsrs	r0, r4, #8
   c:	f7ff fffe 	bl	0 <GLCD_Ustaw_Adres>
D:\STM32\Program\1.11_Odchudzanie\um0427\FWLib\project/t6963c.c:215
  10:	2024      	movs	r0, #36
  12:	f7ff fffe 	bl	0 <GLCD_Ustaw_Adres>
D:\STM32\Program\1.11_Odchudzanie\um0427\FWLib\project/t6963c.c:216
  16:	bd10      	pop	{r4, pc}
Disassembly of section .text.GLCD_Initalize:

00000000 <GLCD_Initalize>:
GLCD_Initalize():
D:\STM32\Program\1.11_Odchudzanie\um0427\FWLib\project/t6963c.c:121
   0:	b570      	push	{r4, r5, r6, lr}
D:\STM32\Program\1.11_Odchudzanie\um0427\FWLib\project/t6963c.c:127
   2:	4c4b      	ldr	r4, [pc, #300]	(130 <GLCD_Initalize+0x130>)
   4:	f44f 7380 	mov.w	r3, #256	; 0x100
D:\STM32\Program\1.11_Odchudzanie\um0427\FWLib\project/t6963c.c:128
   8:	2602      	movs	r6, #2
D:\STM32\Program\1.11_Odchudzanie\um0427\FWLib\project/t6963c.c:129
   a:	2510      	movs	r5, #16
D:\STM32\Program\1.11_Odchudzanie\um0427\FWLib\project/t6963c.c:130
   c:	4849      	ldr	r0, [pc, #292]	(134 <GLCD_Initalize+0x134>)
   e:	4621      	mov	r1, r4
D:\STM32\Program\1.11_Odchudzanie\um0427\FWLib\project/t6963c.c:127
  10:	8023      	strh	r3, [r4, #0]
D:\STM32\Program\1.11_Odchudzanie\um0427\FWLib\project/t6963c.c:128
  12:	70a6      	strb	r6, [r4, #2]
D:\STM32\Program\1.11_Odchudzanie\um0427\FWLib\project/t6963c.c:129
  14:	70e5      	strb	r5, [r4, #3]
D:\STM32\Program\1.11_Odchudzanie\um0427\FWLib\project/t6963c.c:130
  16:	f7ff fffe 	bl	0 <GPIO_Init>
D:\STM32\Program\1.11_Odchudzanie\um0427\FWLib\project/t6963c.c:133
  1a:	f64f 73c4 	movw	r3, #65476	; 0xffc4
D:\STM32\Program\1.11_Odchudzanie\um0427\FWLib\project/t6963c.c:136
  1e:	4846      	ldr	r0, [pc, #280]	(138 <GLCD_Initalize+0x138>)
  20:	4621      	mov	r1, r4
D:\STM32\Program\1.11_Odchudzanie\um0427\FWLib\project/t6963c.c:133
  22:	8023      	strh	r3, [r4, #0]
D:\STM32\Program\1.11_Odchudzanie\um0427\FWLib\project/t6963c.c:134
  24:	70a6      	strb	r6, [r4, #2]
D:\STM32\Program\1.11_Odchudzanie\um0427\FWLib\project/t6963c.c:135
  26:	70e5      	strb	r5, [r4, #3]
D:\STM32\Program\1.11_Odchudzanie\um0427\FWLib\project/t6963c.c:136
  28:	f7ff fffe 	bl	0 <GPIO_Init>
D:\STM32\Program\1.11_Odchudzanie\um0427\FWLib\project/t6963c.c:139
  2c:	f04f 03c0 	mov.w	r3, #192	; 0xc0
D:\STM32\Program\1.11_Odchudzanie\um0427\FWLib\project/t6963c.c:142
  30:	4842      	ldr	r0, [pc, #264]	(13c <GLCD_Initalize+0x13c>)
  32:	4621      	mov	r1, r4
D:\STM32\Program\1.11_Odchudzanie\um0427\FWLib\project/t6963c.c:139
  34:	8023      	strh	r3, [r4, #0]
D:\STM32\Program\1.11_Odchudzanie\um0427\FWLib\project/t6963c.c:140
  36:	70a6      	strb	r6, [r4, #2]
D:\STM32\Program\1.11_Odchudzanie\um0427\FWLib\project/t6963c.c:141
  38:	70e5      	strb	r5, [r4, #3]
D:\STM32\Program\1.11_Odchudzanie\um0427\FWLib\project/t6963c.c:142
  3a:	f7ff fffe 	bl	0 <GPIO_Init>
D:\STM32\Program\1.11_Odchudzanie\um0427\FWLib\project/t6963c.c:146
  3e:	483f      	ldr	r0, [pc, #252]	(13c <GLCD_Initalize+0x13c>)
  40:	2180      	movs	r1, #128
  42:	f7ff fffe 	bl	0 <GPIO_ResetBits>
D:\STM32\Program\1.11_Odchudzanie\um0427\FWLib\project/t6963c.c:147
  46:	483d      	ldr	r0, [pc, #244]	(13c <GLCD_Initalize+0x13c>)
  48:	2140      	movs	r1, #64
  4a:	f7ff fffe 	bl	0 <GPIO_ResetBits>
D:\STM32\Program\1.11_Odchudzanie\um0427\FWLib\project/t6963c.c:148
  4e:	483a      	ldr	r0, [pc, #232]	(138 <GLCD_Initalize+0x138>)
  50:	2140      	movs	r1, #64
  52:	f7ff fffe 	bl	0 <GPIO_ResetBits>
D:\STM32\Program\1.11_Odchudzanie\um0427\FWLib\project/t6963c.c:149
  56:	4837      	ldr	r0, [pc, #220]	(134 <GLCD_Initalize+0x134>)
  58:	f44f 7180 	mov.w	r1, #256	; 0x100
  5c:	f7ff fffe 	bl	0 <GPIO_ResetBits>
D:\STM32\Program\1.11_Odchudzanie\um0427\FWLib\project/t6963c.c:150
  60:	4835      	ldr	r0, [pc, #212]	(138 <GLCD_Initalize+0x138>)
  62:	2104      	movs	r1, #4
  64:	f7ff fffe 	bl	0 <GPIO_ResetBits>
D:\STM32\Program\1.11_Odchudzanie\um0427\FWLib\project/t6963c.c:151
  68:	4833      	ldr	r0, [pc, #204]	(138 <GLCD_Initalize+0x138>)
  6a:	2180      	movs	r1, #128
  6c:	f7ff fffe 	bl	0 <GPIO_ResetBits>
D:\STM32\Program\1.11_Odchudzanie\um0427\FWLib\project/t6963c.c:153
  70:	4831      	ldr	r0, [pc, #196]	(138 <GLCD_Initalize+0x138>)
  72:	f44f 417f 	mov.w	r1, #65280	; 0xff00
  76:	f7ff fffe 	bl	0 <GPIO_Write>
D:\STM32\Program\1.11_Odchudzanie\um0427\FWLib\project/t6963c.c:156
  7a:	482f      	ldr	r0, [pc, #188]	(138 <GLCD_Initalize+0x138>)
  7c:	2104      	movs	r1, #4
  7e:	f7ff fffe 	bl	0 <GPIO_SetBits>
  82:	2200      	movs	r2, #0
D:\STM32\Program\1.11_Odchudzanie\um0427\FWLib\project/t6963c.c:160
  84:	bf00      	nop
D:\STM32\Program\1.11_Odchudzanie\um0427\FWLib\project/t6963c.c:159
  86:	4b2e      	ldr	r3, [pc, #184]	(140 <GLCD_Initalize+0x140>)
  88:	3201      	adds	r2, #1
  8a:	429a      	cmp	r2, r3
  8c:	d1fa      	bne.n	84 <GLCD_Initalize+0x84>
D:\STM32\Program\1.11_Odchudzanie\um0427\FWLib\project/t6963c.c:163
  8e:	482a      	ldr	r0, [pc, #168]	(138 <GLCD_Initalize+0x138>)
  90:	2180      	movs	r1, #128
  92:	f7ff fffe 	bl	0 <GPIO_ResetBits>
D:\STM32\Program\1.11_Odchudzanie\um0427\FWLib\project/t6963c.c:167
  96:	2180      	movs	r1, #128
  98:	4827      	ldr	r0, [pc, #156]	(138 <GLCD_Initalize+0x138>)
  9a:	f7ff fffe 	bl	0 <GPIO_SetBits>
D:\STM32\Program\1.11_Odchudzanie\um0427\FWLib\project/t6963c.c:171
  9e:	2080      	movs	r0, #128
  a0:	f7ff fffe 	bl	0 <GLCD_Initalize>
D:\STM32\Program\1.11_Odchudzanie\um0427\FWLib\project/t6963c.c:172
  a4:	2002      	movs	r0, #2
  a6:	f7ff fffe 	bl	0 <GLCD_Initalize>
D:\STM32\Program\1.11_Odchudzanie\um0427\FWLib\project/t6963c.c:173
  aa:	2042      	movs	r0, #66
  ac:	f7ff fffe 	bl	0 <GLCD_Initalize>
  b0:	2200      	movs	r2, #0
D:\STM32\Program\1.11_Odchudzanie\um0427\FWLib\project/t6963c.c:176
  b2:	bf00      	nop
D:\STM32\Program\1.11_Odchudzanie\um0427\FWLib\project/t6963c.c:175
  b4:	4b22      	ldr	r3, [pc, #136]	(140 <GLCD_Initalize+0x140>)
  b6:	3201      	adds	r2, #1
  b8:	429a      	cmp	r2, r3
  ba:	d1fa      	bne.n	b2 <GLCD_Initalize+0xb2>
D:\STM32\Program\1.11_Odchudzanie\um0427\FWLib\project/t6963c.c:179
  bc:	2028      	movs	r0, #40
  be:	f7ff fffe 	bl	0 <GLCD_Initalize>
D:\STM32\Program\1.11_Odchudzanie\um0427\FWLib\project/t6963c.c:180
  c2:	2000      	movs	r0, #0
  c4:	f7ff fffe 	bl	0 <GLCD_Initalize>
D:\STM32\Program\1.11_Odchudzanie\um0427\FWLib\project/t6963c.c:181
  c8:	2043      	movs	r0, #67
  ca:	f7ff fffe 	bl	0 <GLCD_Initalize>
D:\STM32\Program\1.11_Odchudzanie\um0427\FWLib\project/t6963c.c:184
  ce:	2000      	movs	r0, #0
  d0:	f7ff fffe 	bl	0 <GLCD_Initalize>
D:\STM32\Program\1.11_Odchudzanie\um0427\FWLib\project/t6963c.c:185
  d4:	2000      	movs	r0, #0
  d6:	f7ff fffe 	bl	0 <GLCD_Initalize>
D:\STM32\Program\1.11_Odchudzanie\um0427\FWLib\project/t6963c.c:186
  da:	2040      	movs	r0, #64
  dc:	f7ff fffe 	bl	0 <GLCD_Initalize>
D:\STM32\Program\1.11_Odchudzanie\um0427\FWLib\project/t6963c.c:188
  e0:	2028      	movs	r0, #40
  e2:	f7ff fffe 	bl	0 <GLCD_Initalize>
D:\STM32\Program\1.11_Odchudzanie\um0427\FWLib\project/t6963c.c:189
  e6:	2000      	movs	r0, #0
  e8:	f7ff fffe 	bl	0 <GLCD_Initalize>
D:\STM32\Program\1.11_Odchudzanie\um0427\FWLib\project/t6963c.c:190
  ec:	2041      	movs	r0, #65
  ee:	f7ff fffe 	bl	0 <GLCD_Initalize>
D:\STM32\Program\1.11_Odchudzanie\um0427\FWLib\project/t6963c.c:192
  f2:	2002      	movs	r0, #2
  f4:	f7ff fffe 	bl	0 <GLCD_Initalize>
D:\STM32\Program\1.11_Odchudzanie\um0427\FWLib\project/t6963c.c:193
  f8:	2000      	movs	r0, #0
  fa:	f7ff fffe 	bl	0 <GLCD_Initalize>
D:\STM32\Program\1.11_Odchudzanie\um0427\FWLib\project/t6963c.c:194
  fe:	2022      	movs	r0, #34
 100:	f7ff fffe 	bl	0 <GLCD_Initalize>
D:\STM32\Program\1.11_Odchudzanie\um0427\FWLib\project/t6963c.c:197
 104:	2000      	movs	r0, #0
 106:	f7ff fffe 	bl	0 <GLCD_Initalize>
D:\STM32\Program\1.11_Odchudzanie\um0427\FWLib\project/t6963c.c:198
 10a:	2000      	movs	r0, #0
 10c:	f7ff fffe 	bl	0 <GLCD_Initalize>
D:\STM32\Program\1.11_Odchudzanie\um0427\FWLib\project/t6963c.c:199
 110:	2024      	movs	r0, #36
 112:	f7ff fffe 	bl	0 <GLCD_Initalize>
D:\STM32\Program\1.11_Odchudzanie\um0427\FWLib\project/t6963c.c:201
 116:	209c      	movs	r0, #156
 118:	f7ff fffe 	bl	0 <GLCD_Initalize>
D:\STM32\Program\1.11_Odchudzanie\um0427\FWLib\project/t6963c.c:203
 11c:	2080      	movs	r0, #128
 11e:	f7ff fffe 	bl	0 <GLCD_Initalize>
D:\STM32\Program\1.11_Odchudzanie\um0427\FWLib\project/t6963c.c:205
 122:	f7ff fffe 	bl	0 <GLCD_Initalize>
D:\STM32\Program\1.11_Odchudzanie\um0427\FWLib\project/t6963c.c:206
 126:	f7ff fffe 	bl	0 <GLCD_Initalize>
D:\STM32\Program\1.11_Odchudzanie\um0427\FWLib\project/t6963c.c:207
 12a:	f7ff fffe 	bl	0 <GLCD_Initalize>
D:\STM32\Program\1.11_Odchudzanie\um0427\FWLib\project/t6963c.c:208
 12e:	bd70      	pop	{r4, r5, r6, pc}
 130:	00000000 	.word	0x00000000
 134:	40010800 	.word	0x40010800
 138:	40010c00 	.word	0x40010c00
 13c:	40011000 	.word	0x40011000
 140:	000186a0 	.word	0x000186a0
